:10048F000A0A536D6172744D6564696120757361F9
:10049F00676520696E666F726D6174696F6E3A0A77
:1004AF0000206F6620746F74616C2000207061678C
:1004BF00657320757365640A0025206F662070616F
:1004CF0067657320757365640A0045726173696EA1
:1004DF00672E2E2E00444F4E450A00556E6B6E6FE1
:1004EF00776E2065736361706520636F6D6D616EEC
:1004FF00640A000A2320536D6172744D656469614B
:10050F00206C6F676765722066756C6C210A0045F9
:10051F0072726F722070726F6772616D6D696E6744
:08052F002070616765210A00DC
:100003008F828E83E493FD601FB40A083099FDC28A
:100013009975990D3099FDC2998F828E83E493F57A
:09002300990FBF00010E80D822E4
:0B002C00D2B28F90C2B4D2B4C2B22294
:0F0037007F7012002C7590FFC2B7AF90D2B72226
:100046008F178E168D158C14D2B3C2B4E4F590D2E8
:10005600B4C2B4851790D2B4C2B4AF17AE16AD15FC
:10006600AC1478081206878F90D2B4C2B4AF17AE1C
:1000760016AD15AC1478101206878F90D2B4C2B3A1
:010086002257
:10008700D2B5E4FFFE20B50B0FBF00010EBE4EF543
:06009700BF20F2C2B522F9
:10009D00751100751000750F00750E007F007E0044
:1000AD007D027C00AB11AA10A90FA80EC312067613
:1000BD005062E4FF12002CAF11AE10AD0FAC0E125A
:1000CD0000467590FF120087E4F512F513C2B7E5EF
:1000DD0090B4FF03D2B722E59060083099FDC29924
:1000ED00859099D2B70513E51370020512E513B487
:1000FD0010DBE512B402D67A0079007800E5112400
:10010D0001F511EA3510F510E9350FF50FE8350E4B
:05011D00F50E808822B0
:10012200C3EF9410EE64809482500EC2B4E4F59052
:10013200D2B40FBF00010E80E77F1012002C120014
:02014200872212
:10014400751100751000750F00750E007F007E009C
:100154007D027C00AB11AA10A90FA80EC31206766B
:100164005047E4FF12002CAF11AE10AD0FAC0E12CD
:1001740000467590FF120087C2B7E590B4FF0BD21A
:10018400B7AF11AE10AD0FAC0E22D2B77A00790022
:100194007800E5112401F511EA3510F510E9350F61
:1001A400F50FE8350EF50E80A3AF11AE10AD0FAC10
:0201B4000E2219
:1001B6008F158E148D138C12E4F51E7B0A7A007946
:1001C600007800AF15AE14AD13AC121205CEAF0316
:1001D6007416251EF8A607AF15AE14AD13AC127B28
:1001E6000A7A00790078001205CE8F158E148D13C9
:1001F6008C12051EEC4D4E4F70C1AF1E151EEF60E2
:10020600113099FDC2997416251EF8E62430F59929
:0302160080E8225B
:100219008F118E108D0F8C0E7E047F8F120003AF0D
:1002290011AE10AD0FAC0E1201B67E047FB01200F4
:10023900037F007E007D027C001201B67E047FBB35
:10024900120003AF11AE10AD0FAC0E7B647A0079CA
:100259000078001205438F118E108D0F8C0E7B00D4
:100269007A00790278001205CE8F118E108D0F8CCD
:0C0279000E1201B67E047FC812000322A2
:100285007E047FD9120003E4FDFC7F6012002CD2AE
:10029500B3C2B4AF058F90D2B4C2B4ECF590D2B46A
:1002A500C2B4EDAE047810CEC313CE13D8F9F590D1
:1002B500D2B4C2B37FD012002C120087120037EFE0
:1002C50030E0083099FDC2997599780DBD00010C93
:1002D500E4B505B6ECB410B27E047FE41200032247
:1002E50075985053877F5389CF438920758DFDD2EB
:1002F5008ED299C2B2C2B3D2B4D2B7D2B57590FF7D
:10030500C2B57FFF12002C1200871201448F0D8E9B
:100315000C8D0B8C0AD2B5E4F508F509C2003098AE
:10032500FDC298E599B44004D20080F22000030292
:1003350003F6C2B5AF99EF24BB70030203C524FCD5
:1003450070030203DB24F96045240A60030203E815
:10035500438780758DFFE50945086022AF09AE0822
:100365001201227A0079007800E50D2401F50DEAE5
:10037500350CF50CE9350BF50BE8350AF50A1200D5
:100385009D53877F758DFDE4F508F509805CE509CA
:1003950045086022AF09AE081201227A007900787B
:1003A50000E50D2401F50DEA350CF50CE9350BF5E5
:1003B5000BE8350AF50A12009DE4F508F509802ACF
:1003C500120285750D00750C00750B00750A00E4A9
:1003D500F508F5098014AF0DAE0CAD0BAC0A120291
:1003E5001980077E047FEA120003D2B5C20002031A
:1003F500233099FDC2998599997F007E007D027C05
:1004050000AB0DAA0CA90BA80AC3120660700A7EE0
:10041500057F02120003020323C2B5E509450870F2
:10042500137F8012002CAF0DAE0CAD0BAC0A120081
:1004350046120087C2B4859990D2B40509E50970C2
:10044500020508E50964107004E508640270357F4B
:100455001012002CF508F509120087120037EF304D
:10046500E0077E057F1E1200037A0079007800E51B
:100475000D2401F50DEA350CF50CE9350BF50BE806
:0A048500350AF50AD2B5020323225E
:03000000020537BF
:0C053700787FE4F6D8FD7581200202E513
:10054300E88FF0A4CC8BF0A42CFCE98EF0A42CFC57
:100553008AF0EDA42CFCEA8EF0A4CDA8F08BF0A4D5
:100563002DCC3825F0FDE98FF0A42CCD35F0FCEB34
:100573008EF0A4FEA9F0EB8FF0A4CFC5F02ECD39F9
:0F058300FEE43CFCEAA42DCE35F0FDE43CFC2266
:1005920075F008758200EF2FFFEE33FECD33CDCC20
:1005A20033CCC58233C5829BED9AEC99E5829840A3
:1005B2000CF582EE9BFEED9AFDEC99FC0FD5F0D680
:1005C200E4CEFBE4CDFAE4CCF9A88222B800C1B9AA
:1005D2000059BA002DEC8BF084CFCECDFCE5F0CBE8
:1005E200F97818EF2FFFEE33FEED33FDEC33FCEB21
:1005F20033FB10D703994004EB99FB0FD8E5E4F9DC
:10060200FA227818EF2FFFEE33FEED33FDEC33FCC8
:10061200C933C910D7059BE99A4007EC9BFCE99ABC
:10062200F90FD8E0E4C9FAE4CCFB2275F010EF2F01
:10063200FFEE33FEED33FDCC33CCC833C810D70701
:100642009BEC9AE899400AED9BFDEC9AFCE899F83C
:0E0652000FD5F0DAE4CDFBE4CCFAE4C8F922CF
:10066000EB9FF5F0EA9E42F0E99D42F0EC6480C811
:0606700064809845F022B1
:10067600EB9FF5F0EA9E42F0E99D42F0E89C45F0DA
:010686002251
:10068700E8600FECC313FCED13FDEE13FEEF13FF51
:03069700D8F12275
:00000001FF
